:100000000C94AD060C94F1060C94F1060C94F106D8
:100010000C94F1060C94F1060C94F1060C94F10684
:100020000C94F1060C94F1060C9405120C94D71262
:100030000C94F1060C94F1060C94F1060C94F10664
:100040000C94F1060C94AF2B0C94F1060C94F10671
:100050000C94F1060C94B6210C94F1060C94F10664
:100060000C94F1060C94F1060C94F1060C94F10634
:100070000C94F1060C94F1060C94F1060C94F10624
:100080000C94F1060C94F1060C94F1060C94F10614
:100090000C94F1060C94F1060C94F1060C94F10604
:1000A0000C94F1060C94F1060C94F1063C135E13CB
:1000B00049145E134914A013C313491418142B14C4
:1000C00079177917A717A717EA172618271A271AD3
:1000D0003E18271A35193519011A271A271A151A21
:1000E00023024C003900E100640000001E001400EF
:1000F00004001D714A0039001F001A0016001B730E
:100100004E002A0020000800070006744B002B0058
:1001100021001500090019004D006400220017009D
:100120000A00050000006574AE0001540000007F65
:100130000000E300AB000154000000770000E20083
:1001400023001C000B00110000002971240018007E
:100150000D0010005000E60025000C000E003600D7
:1001600051002800260012000F00370052002C001A
:1001700027001300330038004F0031002D002F00FE
:100180003400E50029000000010001000100010029
:10019000010000003A000100F700FB00010001002F
:1001A0003B00F400F200FA00FD00F5003C00F00016
:1001B000F100F900FE00F4003D00F500F300FC0042
:1001C000FF0001003E000100F800F6000000010001
:1001D0000100010000000100000001000100010019
:1001E00000000100000001003F0001000100B40018
:1001F000000001004000AA00AC00B60001000100B0
:100200004100A800AD00B5000100B7004200A90000
:10021000AE00B9000100B60043000100AB00B7001A
:100220000100010044004500010001000100000040
:100230000A002530313662003A200025303258005D
:100240000A722F6320303132333435363738394132
:1002500042434445460A000A002530325800626F86
:10026000756E6365213A20006C656674207369645D
:10027000652061747461636865640A006C65667406
:100280002073696465206E6F7420726573706F6E81
:1002900064696E670A00747279696E6720746F20F2
:1002A0007265736574206D637032333031380A00C3
:1002B0000A44454255473A20656E61626C65642E7A
:1002C0000A005B735D004B6579626F617264207335
:1002D000746172742E0A005B575D005B535D005BB6
:1002E000525D005B445D005B435D00160345007298
:1002F0000067006F0044006F007800200045005A3E
:1003000000000016034500720067006F0044006F94
:10031000007800200045005A000000040309040989
:10032000028D00050100A0FA09040000010301018B
:1003300000092111010001223F0007058103080087
:100340000A09040100010301020009211101000151
:10035000224D000705820308000A09040200010378
:100360000000000921110100012236000705830366
:1003700008000A090403000203000000092111011A
:100380000001222000070584032000010705040363
:1003900020000109040400010300000009211101EB
:1003A0000001223900070585031000011201100128
:1003B00000000008EDFE0713010001020001050125
:1003C0000906A101050719E029E71500250195088F
:1003D000750181020508190129059505750191022C
:1003E000950175039101050719002977150025016D
:1003F000957875018102C00631FF0974A101097564
:10040000150025FF9520750881020976150025FF46
:10041000952075089102C005010980A10185021689
:10042000010026B7001A01002AB700751095018156
:1004300000C0050C0901A1018503160100269C02DC
:100440001A01002A9C02751095018100C00501095E
:1004500002A1010901A100050919012905150025BD
:100460000195057501810295017503810105010959
:100470003009311581257F950275088106093815E7
:1004800081257F950175088106050C0A38021581C2
:10049000257F950175088106C0C005010906A101E7
:1004A000050719E029E71500250195087501810266
:1004B0009501750881010508190129059505750142
:1004C00091029501750391010507190029FF150097
:1004D00025FF950675088100C00A00253032582096
:1004E000006B6579626F6172645F7265706F7274C0
:1004F0003A20000A0025303258006B6579626F613E
:1005000072645F7365745F6C65643A200064656C47
:100510005F6B65795F6269743A2063616E2774204E
:1005200064656C3A20253032580A006164645F6B60
:1005300065795F6269743A2063616E277420616433
:10054000643A20253032580A00646F6E652E0A0026
:10055000626F6F676D61676963207363616E3A20D4
:100560002E2E2E2000290A002575002F002575004B
:100570005D2800256400200025640020002564001B
:1005800020002564007C0025303258006D6F7573A3
:10059000656B6579205B62746E7C782079207620AB
:1005A000685D287265702F61636C293A205B006D6D
:1005B0006B5F776865656C5F74696D655F746F5FAD
:1005C0006D6178203D2025640A006D6B5F7768655A
:1005D000656C5F6D61785F7370656564203D202593
:1005E000640A006D6B5F74696D655F746F5F6D6148
:1005F00078203D2025640A006D6B5F6D61785F7324
:1006000070656564203D2025640A006D6B5F696E2E
:1006100074657276616C203D2025640A006D6B5F05
:1006200064656C6179203D2025640A006D6B5F77FD
:100630006865656C5F74696D655F746F5F6D617827
:10064000203D2025640A006D6B5F776865656C5FEF
:100650006D61785F7370656564203D2025640A00D4
:100660006D6B5F74696D655F746F5F6D6178203D60
:100670002025640A006D6B5F6D61785F737065653E
:1006800064203D2025640A006D6B5F696E7465729D
:1006900076616C203D2025640A006D6B5F64656C9B
:1006A0006179203D2025640A000A00257500363A4C
:1006B00020776865656C5F74696D655F746F5F6DE9
:1006C00061783A20000A00257500353A2077686580
:1006D000656C5F6D61785F73706565643A20000AD0
:1006E00000257500343A2074696D655F746F5F6D25
:1006F00061783A20000A00257500333A206D617850
:100700005F73706565643A20000A00257500323A0F
:1007100020696E74657276616C286D73293A2000C9
:100720000A00257500313A2064656C6179282A3108
:10073000306D73293A20000A092D2056616C7565C9
:1007400073202D0A004D3E004D25643E20003F00E1
:100750007365742064656661756C740A00433E209D
:100760000077686572652064656C74613A20637512
:1007700072736F723D25642C20776865656C3D252A
:10078000640A53656520687474703A2F2F656E2E65
:1007900077696B6970656469612E6F72672F77691D
:1007A0006B692F4D6F7573655F6B6579730A000A0E
:1007B000092D204D6F7573656B6579202D0A4553A2
:1007C000432F713A09717569740A313A0964656C8D
:1007D0006179282A31306D73290A323A09696E74B9
:1007E000657276616C286D73290A333A096D6178F8
:1007F0005F73706565640A343A0974696D655F7486
:100800006F5F6D61780A353A09776865656C5F6D71
:1008100061785F73706565640A363A097768656563
:100820006C5F74696D655F746F5F6D61780A0A70E3
:100830003A097072696E742076616C7565730A642A
:100840003A097365742064656661756C74730A7522
:10085000703A092B310A646F776E3A092D310A70AC
:100860006775703A092B31300A7067646F776E3A9A
:10087000092D31300A0A7370656564203D20646576
:100880006C7461202A206D61785F737065656420E7
:100890002A2028726570656174202F2074696D6547
:1008A0005F746F5F6D6178290A003F004D3E200044
:1008B000433E20004C25640A000A092D20436F6E38
:1008C000736F6C65202D0A4553432F713A0971757A
:1008D00069740A6D3A096D6F7573656B65790A0005
:1008E0000A092D204D61676963202D0A643A096465
:1008F000656275670A783A096465627567206D619B
:10090000747269780A6B3A096465627567206B6571
:1009100079626F6172640A6D3A0964656275672075
:100920006D6F7573650A763A0976657273696F6ED5
:100930000A733A097374617475730A633A09636FD1
:100940006E736F6C65206D6F64650A302D343A09E3
:100950006C61796572302D34284631302D4634294A
:100960000A506175733A09626F6F746C6F616465E8
:10097000720A653A09656570726F6D0A6E3A094EC2
:100980004B524F0A7A3A09736C656570204C4544A6
:1009900020746573740A000A002575002E6E6B7250
:1009A0006F3A20000A002575002E737761705F6230
:1009B00061636B736C6173685F6261636B737061B9
:1009C00063653A20000A002575002E737761705F19
:1009D00067726176655F6573633A20000A0025756A
:1009E000002E6E6F5F6775693A20000A002575005A
:1009F0002E737761705F72616C745F726775693AAC
:100A000020000A002575002E737761705F6C616CA1
:100A1000745F6C6775693A20000A002575002E63C3
:100A20006170736C6F636B5F746F5F636F6E747212
:100A30006F6C3A20000A002575002E737761705F95
:100A4000636F6E74726F6C5F636170736C6F636BF6
:100A50003A20000A0025303258006B65796D6170CC
:100A60005F636F6E6669672E7261773A20000A00D5
:100A70002575002E6D6F7573653A20000A00257587
:100A8000002E6B6579626F6172643A20000A00255E
:100A900075002E6D61747269783A20000A00257520
:100AA000002E656E61626C653A20000A00253032C6
:100AB000580064656275675F636F6E6669672E7262
:100AC00061773A20000A0025750064656661756CDF
:100AD000745F6C617965723A20003F004E4B524F53
:100AE0003A206F66660A004E4B524F3A206F6E0AEC
:100AF0000074696D65725F636F756E743A2025309E
:100B0000346C580A006B6579626F6172645F6E6B5A
:100B1000726F3A2025580A006B6579626F617264C2
:100B20005F69646C653A2025580A006B6579626FCD
:100B30006172645F70726F746F636F6C3A202558D6
:100B40000A00686F73745F6B6579626F6172645FCE
:100B50006C65647328293A2025580A000A092D205B
:100B6000537461747573202D0A004743433A20344F
:100B70002E382E32204156522D4C4942433A2031D4
:100B80002E382E30204156525F415243483A206160
:100B90007672350A004F5054494F4E533A204C5507
:100BA000464120424F4F544D41474943204D4F55F8
:100BB00053454B45592045585452414B45592043C4
:100BC0004F4E534F4C4520434F4D4D414E44204EC8
:100BD0004B524F203531320A004255494C443A209D
:100BE000376638346162362D646972747920283032
:100BF000333A33303A3338204A616E203232203271
:100C0000303136290A005649443A20307846454565
:100C100044284572676F446F7820455A292050490F
:100C2000443A20307831333037284572676F446F4B
:100C30007820455A29205645523A203078303030B5
:100C4000310A00444553433A20742E6D2E6B2E20FA
:100C50006B6579626F617264206669726D7761722B
:100C60006520666F72204572676F646F780A000AAC
:100C7000092D2056657273696F6E202D0A000A6D6A
:100C80006F7573653A206F66660A000A6D6F75733B
:100C9000653A206F6E0A000A6B6579626F61726453
:100CA0003A206F66660A000A6B6579626F6172644A
:100CB0003A206F6E0A000A6D61747269783A206F8B
:100CC00066660A000A6D61747269783A206F6E0A6E
:100CD000000A64656275673A206F6E0A000A6465EF
:100CE0006275673A206F66660A000A0A626F6F745F
:100CF0006C6F616465722E2E2E2000433E200065CD
:100D000065636F6E6669673A0A00536C65657020AB
:100D10004C454420746573740A0000000000000014
:100D20000000000000010204060A0F17202C3A4AB6
:100D30005D71879DB3C7DAE9F5FCFFFCF5E9DAC719
:100D4000B39D87715D4A3A2C20170F0A06040201F1
:100D50000000000000000000000011241FBECFEFC3
:100D6000DAE0DEBFCDBF04B603FE24C08091F901F6
:100D70009091FA01A091FB01B091FC018730904B5A
:100D8000A740B04BB9F41092F9011092FA011092F9
:100D9000FB011092FC0114BE84B7877F84BF88E1F9
:100DA0000FB6F89480936000109260000FBEE0E0F0
:100DB000FFE3099511E0A0E0B1E0EAEFFAE502C037
:100DC00005900D92AA33B107D9F711E0AAE3B1E07B
:100DD00001C01D92A93FB107E1F70E943F0F0C949B
:100DE0007B2D0C940000FF93EF93E0913A01F0917A
:100DF0003B01309709F00995EF91FF910895FC01AF
:100E00008591803011F0EFDFFBCF0895FF27E0E2FE
:100E100030E247FF0CC0419597FF09C0EDE26095B5
:100E2000709580959095611D711D811D911D27FF05
:100E300002C0219530E350E2AA27660F771F881F72
:100E4000991FAA1FA41710F0A41B63955A95A9F720
:100E5000AA3008F0A95FA05DAF93F3956115710505
:100E60008105910541F7ED3211F4EF93F395F217F7
:100E700018F43F93F395FBCF8F91B5DFFA95E1F727
:100E80000895E991F9918591803021F0853219F02A
:100E9000AADFF9CF089520E0E89455915532C1F3C7
:100EA000503311F4689455915A3348F4505390F3E9
:100EB000220F022E220F220F200D250FF4CF0EF449
:100EC000219589919991533619F3533729F1533567
:100ED00059F1BC0188279927E8945C3621F489915F
:100EE000999168945591543639F446EF7EF077FF26
:100EF0000DC08FEF9FEF0AC055374AE039F05835E3
:100F000040E121F0523642E009F00895FF93EF935B
:100F10007DDFEF91FF91B7CFFF93EF93FC018191BC
:100F20008030B9F360DFFBCFFF93EF9368DFF1CF41
:100F3000DF93CF93CDB7DEB72596A3DFCF91DF91B7
:100F4000089561110BC0FC018281882321F085EE98
:100F50000E940D1603C085EE0E94D51680E090E039
:100F6000089508956091BC017091BD018091BE010A
:100F70009091BF010E94BA2056985E9825982D98AE
:100F800026982E9827982F98813019F4269A2E9A11
:100F9000089556985E98089582EB97E0892B11F09A
:100FA0000E94B20780E090E0089556985E982598D8
:100FB0002D9826982E9827982F988FEF90E0909351
:100FC00089008093880090938B0080938A0090938F
:100FD0008D0080938C00259A2D9A2FEF80E792E068
:100FE000215080409040E1F700C00000269A2E9AE0
:100FF0002FEF80E792E0215080409040E1F700C061
:101000000000279A2F9A2FEF80E792E0215080402E
:101010009040E1F700C0000025982D982FEF80E761
:1010200092E0215080409040E1F700C000002698F7
:101030002E982FEF80E792E0215080409040E1F71A
:1010400000C0000027982F9856985E9825982D98F4
:1010500026982E9827982F98089589EA80938000E3
:1010600089E08093810024982C983F988AB18F74EE
:101070008AB96E98479A8BB1806B8BB9769A0E9429
:10108000D50781EB97E0892B11F00E94B10780E032
:1010900090E0089580E28093000180913C018111ED
:1010A0000EC00E94990881E080933C012FEF83EDF0
:1010B00090E3215080409040E1F700C0000080E4C0
:1010C0000E949F088093000181112EC00E94C908D0
:1010D00080930001811128C00E94C90880930001FB
:1010E000811122C08FE30E94C90880930001811101
:1010F0001BC00E94C10880E40E949F0880930001E9
:10110000811112C08CE00E94C908809300018111F6
:101110000BC00E94C90880930001811105C08FE3B4
:101120000E94C908809300010E94C10880910001BB
:1011300008951092B9008AE08093B800089594EA67
:101140009093BC009091BC0097FFFCCF9091B900A8
:10115000987F983021F0903111F081E008958093CC
:10116000BB0084E88093BC008091BC0087FFFCCF6B
:101170008091B900887F883111F0803471F780E068
:10118000089584E98093BC008091BC0084FDFCCF6D
:1011900008958093BB0084E88093BC008091BC00DC
:1011A00087FFFCCF9091B900987F81E0983209F4D5
:1011B00080E0089584E88093BC008091BC0087FFA4
:1011C000FCCF8091BB00089580910001811115C072
:1011D00080E40E949F088093000181110CC082E18D
:1011E0000E94C90880930001811105C08FEF0E9401
:1011F000C908809300010E94C10884B1807F84B92E
:1012000085B1807F85B98AB1837F8AB98BB1837FAD
:101210008BB93E98469808950E944A088093000131
:101220000E94E40880B38C7080BB81B3836F81BB64
:10123000ECE4F1E0AEE3B1E011921D9281E0EA3519
:10124000F807D1F78DE298E0892B11F00C942D0866
:1012500008959F92AF92BF92CF92DF92EF92FF924A
:101260000F931F93CF93DF93809100018823E1F0C8
:1012700080913D018F5F80933D01811115C086E90A
:1012800092E00E94FF060E944A0880930001882392
:1012900029F08CE792E00E94FF0606C088E692E003
:1012A0000E94FF060E94D5070EE311E0C0E0D0E0E7
:1012B000BB24B39482E0A82ECC24C394D12C29E57E
:1012C000E22E22E0F22EC73000F58091000181115C
:1012D00062C080E40E949F0880930001811112C0C7
:1012E00082E10E94C9088093000181110BC0C601F0
:1012F0000C2E01C0880F0A94EAF780950E94C90855
:10130000809300010E94C10846C0CA30A1F028F4B1
:10131000C83059F0C93061F005C0CC3089F070F0A8
:10132000CD3089F0209A289810C0219A29980DC0B4
:10133000229A2A980AC0239A2B9807C0529A01C071
:10134000539A5B9802C03E9A4698E0EAEA95F1F714
:101350008FB1799985C092E081708B25892B7C9B18
:1013600002C090E001C094E0892B7D9B02C090E018
:1013700001C098E0892B7E9B02C090E001C090E103
:10138000892B9FB19095991F9927991F9295990F35
:10139000907E892B10C080910001811176C080E47D
:1013A0000E949F0880930001882309F45BC0912C60
:1013B0000E94C108892DF8019081981739F1808326
:1013C00080910101882301F18091D70180FF04C041
:1013D0008EE592E00E94FF068091D70180FF0CC04D
:1013E000809101011F928F93FF92EF920E949807C4
:1013F0000F900F900F900F908091D70180FF04C045
:1014000087E592E00E94FF06A09201010E94E40895
:1014100021960F5F1F4FCE30D10509F054CF809138
:1014200001018823B1F0815080930101882339F0B4
:101430008FE99FE00197F1F700C000000AC0ACE41B
:10144000B1E0EEE3F1E081918D9391E0EC34F907A6
:10145000D1F78CEC97E0892BD1F00E94CC0717C014
:1014600090E07ACF83E10E94C90880930001811146
:101470009ECF81E40E949F0880930001811197CF45
:101480000E94DA08982E909493CF80E094CF81E068
:10149000DF91CF911F910F91FF90EF90DF90CF9050
:1014A000BF90AF909F900895E82FF0E0E45BFE4F6F
:1014B00080810895CF92DF92EF92FF920F931F9356
:1014C000CF93DF9380E492E00E94FF063CE4E32E9A
:1014D00031E0F32EC0E0D0E04BE3C42E42E0D42E46
:1014E00002E312E0DF93CF93DF92CF920E9498073E
:1014F00088E392E00E94FF06F70181917F0190E06E
:101500000E941F219F938F931F930F930E94980710
:1015100080E392E00E94FF0621968DB79EB7089661
:101520000FB6F8949EBF0FBE8DBFCE30D105D1F659
:10153000DF91CF911F910F91FF90EF90DF90CF90AF
:1015400008958B3B910578F4883A910540F5853AEA
:101550009105D0F48430910508F0B1C08130910537
:1015600009F4ADC06BC0803E910508F467C0883EA9
:10157000910508F4A4C09C01205F31092031310598
:1015800008F05CC090650895853A910509F459C04A
:10159000863A910509F458C083E890E40895883AA2
:1015A000910509F454C0893A910509F453C08A3A67
:1015B000910509F452C08B3A910509F451C08C3A57
:1015C000910509F450C08D3A910509F44FC0803B54
:1015D000910509F44EC08E3A910509F44DC08F3A39
:1015E000910509F44CC0813B910509F44BC0823B45
:1015F000910509F44AC0833B910509F449C0843B35
:10160000910509F448C0853B910509F447C0863B24
:10161000910509F446C0873B910509F445C0883B14
:10162000910509F444C0893B910509F443C08A3B04
:10163000910509F042C08AE296E4089580E090E0C6
:10164000089581E890E4089582E890E4089582EE98
:1016500094E4089589EE94E408958AEE94E408955C
:1016600085EB94E4089586EB94E4089587EB94E485
:1016700008958CEC94E408958DEC94E4089583E847
:1016800095E408958AE895E4089582E995E408953B
:1016900084E995E4089581E296E4089583E296E46E
:1016A000089584E296E4089585E296E4089586E23A
:1016B00096E4089587E296E4089580E094E408951E
:1016C000089596E0799FF001112494E5899FE00D3B
:1016D000F11D1124E60FF11DEE0FFF1FE052FF4F29
:1016E000859194910895880F991F805A9040FC012C
:1016F000859194910895880F991F80529F4FFC0106
:1017000085919491089526E0729FF001112444E59B
:10171000849FE00DF11D1124E60FF11DEE0FFF1F58
:10172000E052FF4F25913491C9019A9581159F414F
:1017300010F4C9010895C90190528115904128F40F
:10174000C9019F700E947B0B0895C90190538115B8
:10175000904120F4C9019927906C0895211580E5E6
:10176000380769F40E94481A9FEF24E34CE0915037
:1017700020404040E1F700C000000C94DB21213004
:1017800080E5380751F480EB92E00E94FF068091DB
:10179000D70181608093D7010895C90190558115C3
:1017A000904108F050C0832F99278F70992781307E
:1017B0009105D9F4A9014370552702C0880F991FDC
:1017C0004A95E2F79C68A90164E0440F551F6A95A9
:1017D000E1F744275370842B952B73E0220F331FBE
:1017E0007A95E1F7207633271DC08230910529F4E0
:1017F000922F8827816F906A089583309105A9F40C
:10180000A9014370552781E090E002C0880F991F1D
:101810004A95E2F79C6843E0220F331F4A95E1F7AF
:10182000207E3770822B932B08950497F1F4A90141
:101830004370552781E090E002C0880F991F4A95B8
:10184000E2F79A68E8CFC90190578115904120F4DA
:10185000C9019F7090620895C90190588115904107
:1018600020F4C9019F70906A0895203E3105E0F48C
:10187000203C310558F52133310509F470C048F496
:101880002932310509F464C02A32310509F46EC0E9
:1018900074C029333105F1F022383105D9F02533F0
:1018A000310509F44EC069C0233E310589F138F491
:1018B000203E3105C1F0223E3105E1F05EC0263EFA
:1018C000310569F1273E3105A9F157C0C9010E94D0
:1018D000730B08958091EA0180FD02C081FF4DC025
:1018E00080EE90E04BC08091EA0180FFF9CF89E360
:1018F00090E044C08091EA0182FF0EC08091EA012D
:1019000084FF03C080E090E039C083EE90E036C0F1
:101910008091EA0182FFF2CF82EE90E02FC08091A9
:10192000EA0183FF0BC08091EA0184FDEBCF87EED3
:1019300090E024C08091EA0183FFF5CF86EE90E02D
:101940001DC08091EA0185FF07C089E290E016C0C2
:101950008091EA0185FFF9CF85E390E00FC0809187
:10196000EA0186FF07C08AE290E008C08091EA01A0
:1019700086FFF9CF81E390E001C0C9010E94A10A6E
:101980000895089580916D0108959FB7F89410927D
:101990005C019FBF9091F001943009F058C0909184
:1019A000E9009F702091EC0020FF02C020E801C0F8
:1019B00020E0292B94E09093E9009091EB0090FFB8
:1019C00043C09091EE0097FF3FC090915A01992338
:1019D00021F09091E80095FF37C010925A0196E0EF
:1019E0003091E80035FD15C03091F001343061F5DB
:1019F0003091EB0035FD28C0915021F481E08093B7
:101A00005A0122C0EFE9FFE03197F1F700C0000072
:101A1000E7CF8093F1008091E80085FD0AC08091B6
:101A2000E80080FFFCCF8091E8008E778093E8008B
:101A300006C08FB7F89491E090935C018FBF2F7030
:101A40002093E90080E008952F702093E9008FEF44
:101A50000895CF93DF9300D01F92CDB7DEB72091CA
:101A6000F001243019F523E029839B838A83209396
:101A7000E9008FEF9091E800815095FD06C095ED4B
:101A80009A95F1F700008111F5CF8091E80085FF6C
:101A90000DC040E050E063E070E0CE0101960E948E
:101AA000F80F8091E8008E778093E8000F900F90F8
:101AB0000F90DF91CF910895CF93DF9300D01F92C5
:101AC000CDB7DEB72091F001243021F522E0298343
:101AD0009B838A8383E08093E9008FEF9091E800F5
:101AE000815095FD06C095ED9A95F1F700008111A2
:101AF000F5CF8091E80085FF0DC040E050E063E045
:101B000070E0CE0101960E94F80F8091E8008E7778
:101B10008093E8000F900F900F90DF91CF91089580
:101B20002091F0012430F1F422E02093E9002FEF1E
:101B30003091E800215035FD06C035ED3A95F1F7BA
:101B400000002111F5CF2091E80025FF0BC040E0F7
:101B500050E065E070E00E94F80F8091E8008E7719
:101B60008093E8000895CF93DF93EC018091F0011A
:101B7000843009F047C080910C018823E1F0809106
:101B80000D018823C1F085E08093E9008FEF9091EB
:101B9000E800815095FD06C095E19A95F1F70000A7
:101BA0008111F5CF8091E80085FF2CC040E050E026
:101BB00060E170E017C081E08093E9008FEF9091C1
:101BC000E800815095FD06C095ED9A95F1F700006B
:101BD0008111F5CF8091E80085FF14C040E050E00E
:101BE00068E070E0CE010E94F80F8091E8008E77E7
:101BF0008093E80080E1FE01ADE5B1E001900D9237
:101C00008A95E1F7DF91CF91089587EE92E00E94E7
:101C1000FF068091EF01811109C00E948A110E9484
:101C2000E7118091E20084608093E200089583EEE2
:101C300092E00E94FF061092EF0108958FED92E06E
:101C40000C94FF068BED92E00E94FF060C949C2BF7
:101C500087ED92E00E94FF060E9476210E94A22B4F
:101C60000E9483140C94C10C80915B018F5F809360
:101C70005B0162E30E94102D911135C010925B014F
:101C800080915C01882379F18091F001843049F5DD
:101C90008091E9008F709091EC0090FF02C090E875
:101CA00001C090E0982B84E08093E9008091EB00E4
:101CB00080FF14C08091EE0087FF10C08091E80083
:101CC00085FF03C01092F100F9CF8091E80080FFFA
:101CD00005C08091E8008E778093E8009F70909314
:101CE000E90010925C01089542E061EC81E00E94FD
:101CF000041142E061EC82E00E94041142E061ECD8
:101D000083E00E94041142E261EC84E00E9404112D
:101D100042E161EC85E00C9404118091F201833082
:101D200009F455C030F4813071F0823009F48EC06E
:101D300008958A3009F47AC08B3009F460C0893084
:101D400009F09CC020C08091F101813A09F096C051
:101D50008091E800877F8093E8008091F501909161
:101D6000F601892B21F060E080E090E003C060E1A3
:101D70008DE591E070E00E9441108091E8008B7742
:101D80008093E80008958091F101813209F076C0D6
:101D90008091F5019091F601009719F0049709F0F0
:101DA0006DC08091E800877F8093E8008091E80013
:101DB00082FD05C08091F0018111F8CF5FC0809154
:101DC000F10080936D018091E8008B7753C0809182
:101DD000F101813A09F052C08091F5019091F6012C
:101DE000892B09F04BC08091E800877F8093E80041
:101DF0008091E80080FFFCCF80910C0136C080917B
:101E0000F1018132D9F58091F5019091F601892B8C
:101E1000A9F58091E800877F8093E8000E9439113E
:101E20008091F30180930C010C94481A8091F10188
:101E3000813221F58091E800877F8093E8000E943D
:101E400039118091F40180936E0108958091F10120
:101E5000813AA1F48091E800877F8093E800809127
:101E6000E80080FFFCCF80916E018093F1008091AB
:101E7000E8008E778093E8000C943911089584B7B8
:101E8000877F84BF88E10FB6F8948093600010923A
:101E900060000FBE90E080E80FB6F8948093610078
:101EA000909361000FBE0E940C150E948A110E943F
:101EB000E7118091E20084608093E20085EC9CE071
:101EC0000E94B52078940E9461140E940E1582E051
:101ED00091E00E947E140E948A2B86EC92E00E9480
:101EE000FF068091F001853089F482EC92E00E9437
:101EF000FF060E9439218091EE01882391F30E9410
:101F00006121882371F30E94E20FEBCF0E943C1500
:101F1000E8CF292F332723303105A9F06CF4213085
:101F2000310509F442C02230310509F043C08DE883
:101F300090E02FE133E042C021323105C9F0223276
:101F4000310519F137C099278130910541F0823070
:101F5000910541F0892B71F5EBE1F3E005C0E3E079
:101F6000F3E002C0EBEEF2E0849190E09F0126C026
:101F7000653000F5E62FF0E0EE0FFF1FEB5DFE4F42
:101F80002081318189E090E019C0653098F4E62F16
:101F9000F0E0DF01AA0FBB1FA55EBE4F2D913C9163
:101FA000EA5EFE4F808190E009C082E190E02CEA79
:101FB00033E004C080E090E020E030E0FA013183BB
:101FC0002083089580E189BD82E189BD09B400FEC6
:101FD000FDCF8091D8008F7D8093D8008091E00064
:101FE00082608093E0008091E00081FDFCCF089545
:101FF000CF92DF92EF92FF920F931F93CF93DF93D5
:102000007C018B01EA010E945A11811131C0209795
:1020100031F088819981081B190BE80EF91EC12C3B
:10202000D12C0115110519F18091E80085FD14C02E
:102030008091E8008E778093E800209741F08881B6
:1020400099818C0D9D1D9983888385E011C00E9424
:102050005A11882331F30CC0F70181917F018093DD
:10206000F10001501109FFEFCF1ADF0ADACF80E04B
:10207000DF91CF911F910F91FF90EF90DF90CF9064
:1020800008952091F7013091F8012617370748F09D
:102090006115710539F42091E8002E772093E8004E
:1020A00001C0B901FC0120E061157105B9F1809111
:1020B000F001882309F440C0853009F43FC08091C5
:1020C000E80083FD3DC08091E80082FF06C080915A
:1020D000E80082FF26C080E008958091E80080FF3C
:1020E000E3CF2091F3008091F20090E0922B6115F4
:1020F000710551F08830910538F421912093F10059
:10210000615071090196F3CF21E0089709F020E0B2
:102110008091E8008E778093E800C6CF2111C7CF69
:10212000D6CF8091F001882339F0853039F0809145
:10213000E80083FFCCCF04C082E0089583E00895D7
:1021400081E008952091F7013091F80126173707B3
:1021500048F06115710539F42091E8002E7720933D
:10216000E80001C0B901FC0120E061157105C1F171
:102170008091F001882309F441C0853009F440C002
:102180008091E80083FD3EC08091E80082FF06C098
:102190008091E80082FF27C080E008958091E800E8
:1021A00080FFE3CF2091F3008091F20090E0922B2A
:1021B0006115710559F08830910540F42491209300
:1021C000F1003196615071090196F2CF21E0089734
:1021D00009F020E08091E8008E778093E800C5CF79
:1021E0002111C6CFD5CF8091F001882339F08530F9
:1021F00039F08091E80083FFCBCF04C082E00895DE
:1022000083E0089581E00895982F973058F59093D2
:10221000E900981739F07091EC002091ED00509191
:10222000F00003C0242F762F50E021FF19C0309119
:10223000EB003E7F3093EB003091ED003D7F30931B
:10224000ED003091EB0031603093EB007093EC00C7
:102250002093ED005093F0002091EE0027FF07C07F
:102260009F5FD3CF8F708093E90081E0089580E075
:1022700008958091F10187FD05C08091E80080FFFD
:102280000EC012C08091E80082FD05C08091F0016F
:102290008111F8CF08958091E8008B7708C0809174
:1022A000F0018111EACF08958091E8008E77809344
:1022B000E80008958091E4009091E50045E62091C2
:1022C000EC0020FF21C02091E80020FD21C02091DA
:1022D000F001222389F0253089F02091EB0025FDC3
:1022E0000FC02091E4003091E5002817390739F339
:1022F000415041F0C901E3CF82E0089583E00895A1
:1023000081E0089584E008952091E80022FFDFCF66
:1023100080E008950E94F8110E940012E0EEF0E0C3
:10232000808181608083E8EDF0E080818F77808319
:1023300019BCA7EDB0E08C918E7F8C9380818F7E4D
:1023400080831092EF0108950F931F93CF93DF9333
:102350000E94F8110E940012C8EDD0E088818F77AA
:10236000888388818068888388818F7D888319BC71
:102370001092F0011092EC011092EE011092ED011A
:1023800000EE10E0F80180818B7F8083888181607E
:10239000888342E060E080E00E940411E1EEF0E01A
:1023A00080818E7F8083E2EEF0E080818160808397
:1023B000808188608083F80180818E7F808388811E
:1023C00080618883DF91CF911F910F910895E8ED8F
:1023D000F0E080818F7E8083E7EDF0E08081816096
:1023E000808384E082BF81E08093EF010C94A4118C
:1023F000E8EDF0E080818E7F80831092E200089506
:102400001092DA001092E10008951F920F920FB619
:102410000F9211242F933F934F935F936F937F936A
:102420008F939F93AF93BF93EF93FF938091E100BE
:1024300082FF0BC08091E20082FF07C08091E10023
:102440008B7F8093E1000E94340E8091DA0080FF40
:102450001FC08091D80080FF1BC08091DA008E7F62
:102460008093DA008091D90080FF0DC080E189BDA2
:1024700082E189BD09B400FEFDCF81E08093F001C7
:102480000E94050E05C019BC1092F0010E94170EA3
:102490008091E10080FF19C08091E20080FF15C0AB
:1024A0008091E2008E7F8093E2008091E200806163
:1024B0008093E2008091D80080628093D80019BC9C
:1024C00085E08093F0010E94220E8091E10084FF5C
:1024D00030C08091E20084FF2CC080E189BD82E1A0
:1024E00089BD09B400FEFDCF8091D8008F7D809317
:1024F000D8008091E1008F7E8093E1008091E2001E
:102500008F7E8093E2008091E20081608093E20000
:102510008091EC01882311F084E007C08091E300F2
:1025200087FF02C083E001C081E08093F0010E9438
:10253000280E8091E10083FF29C08091E20083FF93
:1025400025C08091E100877F8093E10082E0809345
:10255000F0011092EC018091E1008E7F8093E10008
:102560008091E2008E7F8093E2008091E2008061A2
:102570008093E20042E060E080E00E9404118091DC
:10258000F00088608093F0000E941E0EFF91EF9192
:10259000BF91AF919F918F917F916F915F914F917B
:1025A0003F912F910F900FBE0F901F9018951F9283
:1025B0000F920FB60F9211242F933F934F935F9377
:1025C0006F937F938F939F93AF93BF93CF93EF932B
:1025D000FF93C091E900CF708091EC001092E90068
:1025E0008091F000877F8093F00078940E9413130D
:1025F0001092E9008091F00088608093F000C09311
:10260000E900FF91EF91CF91BF91AF919F918F9191
:102610007F916F915F914F913F912F910F900FBEDE
:102620000F901F9018951F93CF93DF93CDB7DEB710
:10263000AA970FB6F894DEBF0FBECDBFE1EFF1E071
:102640008091F100819321E0E93FF207C9F70E94F0
:102650008D0E8091E80083FF1CC12091F101309123
:10266000F201832F90E08A30910508F012C1FC013D
:10267000EA5AFF4F0C94302D203881F0223809F0AF
:1026800008C18091F5018F708093E9008091EB0083
:1026900085FB882780F91092E90006C08091ED0142
:1026A0009091EE01911182609091E800977F909354
:1026B000E8008093F1001092F100C5C0822F8D7F59
:1026C00009F0E7C0222319F0223061F0E2C08091C6
:1026D000F301813009F0DDC0333009F080E08093F0
:1026E000EE0128C08091F301811124C02091F501F1
:1026F0002F7009F4CEC02093E9008091EB0080FF99
:1027000019C08091EB00333011F4806211C08061F8
:102710008093EB0081E090E0022E01C0880F0A94C4
:10272000EAF78093EA001092EA008091EB0088605B
:102730008093EB001092E9008091E800877F86C0CB
:102740002111A7C01091F3011F778091E3008078D9
:10275000812B8093E3008091E800877F8093E800DD
:102760000E9439118091E80080FFFCCF8091E30046
:1027700080688093E300112311F083E001C082E0C0
:102780008093F00186C02058223008F082C08091EA
:10279000F3019091F4018C3D23E0920779F583E0F9
:1027A0008A838AE289834FB7F894DE01139620E08A
:1027B0003EE051E2E32FF0E050935700E49120FF18
:1027C00003C0E295EF703F5FEF708E2F90E0EA302C
:1027D00010F0C79601C0C0968D939D932F5F243152
:1027E00049F74FBF8091E800877F8093E8006AE255
:1027F00070E0CE0101960E94411014C0AE014F5FFF
:102800005F4F6091F5010E94890F009709F441C064
:102810002091E800277F2093E800BC0189819A81FC
:102820000E94A2108091E8008B778093E80031C06D
:10283000203879F58091E800877F8093E8008091C7
:10284000EC018093F1008091E8008E778093E8009E
:102850000E9439111EC021111CC09091F3019230C9
:10286000C0F48091E800877F8093E8009093EC01AA
:102870000E9439118091EC01811104C08091E30024
:1028800087FF02C084E001C081E08093F0010E94D4
:10289000740E8091E80083FF0AC08091E800877F72
:1028A0008093E8008091EB0080628093EB00AA9611
:1028B0000FB6F894DEBF0FBECDBFDF91CF911F9151
:1028C0000895CF938091F0018823B1F08091E900C1
:1028D0008F709091EC0090FF02C090E801C090E0F2
:1028E000C92FC82B1092E9008091E80083FD0E9457
:1028F0001313CF70C093E900CF91089590937401A2
:10290000809373010895E0917301F0917401309701
:1029100021F00190F081E02D099480E00895FF926C
:102920000F931F93CF93DF938C01E0917301F0918C
:102930007401309799F10280F381E02D099580911F
:10294000D70182FF2BC080FF04C081EE94E00E947B
:10295000FF06E80180E1F82E0BED14E08091D7012D
:1029600080FF0BC088811F928F931F930F930E944B
:1029700098070F900F900F900F90FA942196F110F6
:10298000EDCF8091D70180FF09C089ED94E0DF9100
:10299000CF911F910F91FF900C94FF06DF91CF9183
:1029A0001F910F91FF900895E0917301F0917401D0
:1029B000309721F00480F581E02D0994089520914D
:1029C0007101309172018217930771F09093720137
:1029D00080937101E0917301F0917401309721F0BF
:1029E0000680F781E02D0994089520916F013091C0
:1029F00070018217930771F09093700180936F01BB
:102A0000E0917301F0917401309721F00084F18519
:102A1000E02D0994089508950C940B150E947821D7
:102A20000E940C090C943E22CF93C82F8091D701AD
:102A300082FF1EC080FF04C08AEF94E00E94FF0660
:102A40008091D70180FF0CC01F92CF9325EF34E017
:102A50003F932F930E9498070F900F900F900F9025
:102A60008091D70180FF04C083EF94E00E94FF06AD
:102A70008C2FCF910C94C10CCF92DF92EF92FF92EA
:102A80000F931F93CF93DF93CDB7DEB72B970FB67E
:102A9000F894DEBF0FBECDBF0E94290936E7E32EB2
:102AA00031E0F32E00E010E0C02E802F0E94540A87
:102AB000F701D1907F01D826B1F40F5F1F4F0E3080
:102AC000110591F78FEF89838A831B820E948121F0
:102AD0008160782F9D838C8349815A816B818D81A0
:102AE0000E94DF1541C09091D70191FF04C08B87F0
:102AF0000E945A0A8B8520E030E04D2D50E0922F45
:102B0000BA01022E02C0759567950A94E2F760FF3C
:102B100025C02E83CF82EE24E394F12C02C0EE0C6C
:102B2000FF1C9A95E2F790E08E219F2121E0892BEE
:102B300009F420E028870E9481218160782F9A87FC
:102B400089874E815F8168858A850E94DF15F8013B
:102B5000EA58FE4F80818E25808306C02F5F3F4F4D
:102B60002630310561F6A9CF0E94AC251091750180
:102B70000E9483141817A1F00E948314809375019A
:102B80002B960FB6F894DEBF0FBECDBFDF91CF916D
:102B90001F910F91FF90EF90DF90CF900C94141540
:102BA0002B960FB6F894DEBF0FBECDBFDF91CF914D
:102BB0001F910F91FF90EF90DF90CF900895CF93EA
:102BC000DF93CDB7DEB72B970FB6F894DEBF0FBEFD
:102BD000CDBF4F83588769877A878B87DE0111962F
:102BE00086E0FD0111928A95E9F785E0FE013796AE
:102BF00001900D928A95E1F749815A816B817C8120
:102C00008D819E810E94141D2B960FB6F894DEBF15
:102C10000FBECDBFDF91CF910895CF93C82F8823EA
:102C200009F4C1C0823859F40E94831481FDBBC0ED
:102C300089E30E94B31F0E948F2089E30CC0833870
:102C400079F40E94831480FDAEC083E50E94B31F17
:102C50000E948F2083E50E940420CF910C948F2046
:102C6000843859F40E94831482FD9DC087E40E9439
:102C7000B31F0E948F2087E4EECF8CEF8C0F813A38
:102C800048F48C2F0E94352A81118DC08C2F0E9410
:102C9000B31FE3CF80E28C0F883048F4C77081E027
:102CA00001C0880FCA95EAF70E945620D6CF8BE55F
:102CB0008C0F833078F4C53A29F0C63A31F482E8B3
:102CC00090E005C081E890E002C083E890E0CF91F9
:102CD0000C94DF1488E58C0F833108F064C0C83A87
:102CE00039F1C93A41F1CA3A49F1CB3A51F1CC3AFA
:102CF00059F1CD3A61F1C03B69F1CE3A71F1CF3A69
:102D000079F1C13B81F1C23B89F1C33B91F1C43BF5
:102D100099F1C53BA1F1C63BA9F1C73BB1F1C83B55
:102D2000B9F1C93BC1F1CA3BC9F58AE292E038C0AA
:102D300082EE90E035C089EE90E032C08AEE90E0FD
:102D40002FC085EB90E02CC086EB90E029C087EB8C
:102D500090E026C08CEC90E023C08DEC90E020C089
:102D600083E891E01DC08AE891E01AC082E991E011
:102D700017C084E991E014C081E292E011C083E2BF
:102D800092E00EC084E292E00BC085E292E008C0BF
:102D900086E292E005C087E292E002C080E090E027
:102DA000CF910C94F514CF910895882309F44BC06A
:102DB000823859F40E94831481FF45C089E30E9440
:102DC000B31F0E948F2089E30CC0833871F40E94E6
:102DD000831480FF38C083E50E94B31F0E948F20B8
:102DE00083E50E9404200C948F20843859F40E94BB
:102DF000831482FF28C087E40E94B31F0E948F20A3
:102E000087E4EFCF9CEF980F913A58F390E2980F38
:102E1000983050F4877091E001C0990F8A95EAF7D5
:102E2000892F0E945C20DFCF9BE5980F933020F420
:102E300080E090E00C94DF14885A833120F480E025
:102E400090E00C94F5140895882321F00E945620F8
:102E50000C948F200895882321F00E945C200C940C
:102E60008F200895CF92DF92EF92FF920F931F93DE
:102E7000CF93DF93CDB7DEB728970FB6F894DEBFB8
:102E80000FBECDBF8C0185E0F801DE0111960190E7
:102E90000D928A95E1F7F80140813181F280258118
:102EA00022952F7083819481892B31F03F3F31F43B
:102EB00081E04F3F19F403C081E001C080E080FD54
:102EC000C6C249833A8389819A812F830E94711FE8
:102ED0009E8388870E94701F0E94431E4E81E42FAC
:102EE000E295EF70F0E0E05AFF4F2F8168850C9477
:102EF000302D842F807F142F1F70882311F012959E
:102F0000107FFF2059F0112309F456C2812F6887E2
:102F10000E9466200E948F2068854EC2862F0E94E4
:102F2000D516112309F493C2812F0E946C20289694
:102F30000FB6F894DEBF0FBECDBFDF91CF911F91CA
:102F40000F91FF90EF90DF90CF900C948F20342F53
:102F5000307F842F8F70303211F08295807F66230E
:102F600019F0613019F12CC0FF20B1F0222309F4CF
:102F700094C1213009F091C128960FB6F894DEBFB4
:102F80000FBECDBFDF91CF911F910F91FF90EF90BA
:102F9000DF90CF900C947620222319F0213009F491
:102FA00056C28E830E9479208E818AC1FF2021F033
:102FB000263008F04CC271C1253008F048C280C1EB
:102FC000FF2021F0222309F468C1F6C1222309F46D
:102FD00077C106C2242F26952695237030E021154F
:102FE000310521F021303105C9F031C2FF2021F037
:102FF000862F942F937002C080E090E028960FB641
:10300000F894DEBF0FBECDBFDF91CF911F910F911E
:10301000FF90EF90DF90CF900C94DF14FF2021F011
:10302000862F942F937002C080E090E028960FB610
:10303000F894DEBF0FBECDBFDF91CF911F910F91EE
:10304000FF90EF90DF90CF900C94F514862FFF2027
:1030500019F00E94322402C00E949A2428960FB6CA
:10306000F894DEBF0FBECDBFDF91CF911F910F91BE
:10307000FF90EF90DF90CF900C941F25842F8370EA
:1030800009F076C0F110E3C1262F2295269527700E
:10309000220F220F862F8F70C82ED12CE12CF12CFD
:1030A000022E04C0CC0CDD1CEE1CFF1C0A94D2F7CF
:1030B00064FF10C06FE070E080E090E004C0660F35
:1030C000771F881F991F2A95D2F760957095809574
:1030D000909503C060E070E0CB01242F26952695E3
:1030E0002370422F50E042305105D1F0433051055A
:1030F00059F16C297D298E299F294130510541F1D3
:1031000028960FB6F894DEBF0FBECDBFDF91CF91EA
:103110001F910F91FF90EF90DF90CF900C94681E5D
:103120006C297D298E299F2928960FB6F894DEBF39
:103130000FBECDBFDF91CF911F910F91FF90EF9008
:10314000DF90CF900C94821E0E94681EC701B601CA
:1031500028960FB6F894DEBF0FBECDBFDF91CF919A
:103160001F910F91FF90EF90DF90CF900C944E1E27
:10317000FF2019F0842F817001C08695882309F4FF
:1031800066C1262F229526952770220F220F862FA3
:103190008F70C82ED12CE12CF12C022E04C0CC0C47
:1031A000DD1CEE1CFF1C0A94D2F764FF10C06FE018
:1031B00070E080E090E004C0660F771F881F991FC1
:1031C0002A95D2F7609570958095909503C060E040
:1031D00070E0CB01242F269526952370422F50E0D6
:1031E00042305105D1F04330510559F16C297D2908
:1031F0008E299F294130510541F128960FB6F89448
:10320000DEBF0FBECDBFDF91CF911F910F91FF9019
:10321000EF90DF90CF900C943C1F6C297D298E2974
:103220009F2928960FB6F894DEBF0FBECDBFDF9161
:10323000CF911F910F91FF90EF90DF90CF900C9462
:10324000561F0E943C1FC701B60128960FB6F8947E
:10325000DEBF0FBECDBFDF91CF911F910F91FF90C9
:10326000EF90DF90CF900C94221F603FC9F118F4CB
:10327000603E50F49CC0623F09F461C008F44BC04A
:10328000633F09F470C093C0162F1F70842F8F7195
:10329000FF2099F00E94BB1E812F28960FB6F8944C
:1032A000DEBF0FBECDBFDF91CF911F910F91FF9079
:1032B000EF90DF90CF900C9424170E94DC1E812F9A
:1032C00028960FB6F894DEBF0FBECDBFDF91CF9129
:1032D0001F910F91FF90EF90DF90CF900C942B17E0
:1032E000FF20A9F0253008F0B2C0842F8F712896F6
:1032F0000FB6F894DEBF0FBECDBFDF91CF911F9107
:103300000F91FF90EF90DF90CF900C94011F26302B
:1033100008F09DC0EACFFF20A1F0842F8F7128967E
:103320000FB6F894DEBF0FBECDBFDF91CF911F91D6
:103330000F91FF90EF90DF90CF900C94BB1EFF2079
:1033400061F3842F8F7128960FB6F894DEBF0FBEFD
:10335000CDBFDF91CF911F910F91FF90EF90DF9044
:10336000CF900C94DC1EFF2091F0842F8F71289653
:103370000FB6F894DEBF0FBECDBFDF91CF911F9186
:103380000F91FF90EF90DF90CF900C94A61E28969F
:103390000FB6F894DEBF0FBECDBFDF91CF911F9166
:1033A0000F91FF90EF90DF90CF900C949C1EFF2028
:1033B000A1F0222309F4B1CF862F28960FB6F894F6
:1033C000DEBF0FBECDBFDF91CF911F910F91FF9058
:1033D000EF90DF90CF900C940D16222309F4B1CF1B
:1033E000862F28960FB6F894DEBF0FBECDBFDF91B3
:1033F000CF911F910F91FF90EF90DF90CF900C94A1
:10340000D5164F70C8010E94A10728960FB6F894F0
:10341000DEBF0FBECDBFDF91CF911F910F91FF9007
:10342000EF90DF90CF900C94C11D4F70C80128968B
:103430000FB6F894DEBF0FBECDBFDF91CF911F91C5
:103440000F91FF90EF90DF90CF900C94600B289637
:103450000FB6F894DEBF0FBECDBFDF91CF911F91A5
:103460000F91FF90EF90DF90CF9008950E9473200E
:103470000E9448200E948F200E944D260E941F25F6
:1034800080E090E00E94DF1480E090E00C94F5145E
:103490000E9463200C94361A0E94711F292F2295D6
:1034A0002F7030E02C3031054CF42A3031056CF4AB
:1034B000225031092230310590F407C02C303105FB
:1034C00051F02F30310539F00AC0803E10F0803FB6
:1034D00031F481E0089593FB882780F9089580E016
:1034E0000895CF93DF9300D000D01F92CDB7DEB701
:1034F0000F900F900F900F900F90DF91CF91089544
:10350000CF93DF9300D000D000D0CDB7DEB72696A2
:103510000FB6F894DEBF0FBECDBFDF91CF910895F7
:103520001F93CF93DF93C091840116E080918501B2
:10353000C81799F0D0E01C9FF0011D9FF00D1124D9
:10354000EA57FE4F40815181628173818481958168
:103550000E94801A2196C770E9CFDF91CF911F9109
:1035600008954091B6015091B7016091B8017091F2
:10357000B9018091BA019091BB010C94801ACF934C
:103580008091BB0182958F7009F05FC08091B80176
:10359000882309F45AC020918401A091850160918B
:1035A000B6017091B7018091B9019091BA0131E0F3
:1035B0006F3F09F030E0B32FC6E02A1709F445C089
:1035C000009721F07F3F21F44B2F03C041E001C061
:1035D00040E030E040FD35C0C29FF001C39FF00DD8
:1035E0001124EA57FE4F418174132BC040816413AC
:1035F00028C04281411125C0438154814817590791
:1036000010F441505109481B590B483C5105C8F46E
:103610008091BB018F7080618093BB0186E0829FA7
:10362000F001839FF00D1124E557FE4F80818F70CC
:103630008061808386EB91E00E943217CF910C94D9
:10364000901A2F5F3F4F2770B8CFCF910895CF9238
:10365000DF92EF92FF920F931F93CF93DF93CDB73B
:10366000DEB762970FB6F894DEBF0FBECDBF8C01F8
:1036700085E0F801DE011D9601900D928A95E1F733
:10368000D8014C9111965C91119712966C911297FA
:103690001396ED90FC9014977091B601E091B701EC
:1036A0002091B9013091BA012115310531F0EF3F78
:1036B00031F481E07F3F19F403C081E001C080E074
:1036C000B82FB170CB2E80FD6CC1D090B801DD2039
:1036D00009F4F5C0F091BB01E216F30638F0C7011A
:1036E000821B930B883C910548F09BC02095309538
:1036F0002E0D3F1D283C310508F093C08F2F807F91
:1037000009F052C0E51314C0741312C0D62E611113
:103710000FC0FF70F061F093BB010E94B11A86EBFD
:1037200091E00E9432178091BB01F80185836CC142
:10373000EF2831F05F3F31F481E04F3F19F403C0CF
:1037400081E001C080E080FD03C081E0862701C0E8
:1037500080E0F82FF170FF2E80FF1CC08091840163
:103760002091850136E0821709F428C190E0389F46
:10377000F001399FF00D1124EA57FE4F7181571364
:1037800006C07081471303C07281671303C001969E
:103790008770E9CFD62E662309F436C18091BB012C
:1037A00081608093BB0153C0E51308C0741306C049
:1037B000611104C0D8011596FC93AEC04D875E8799
:1037C0008D859E856A8B0E944C1A6A89882329F10F
:1037D000D62E662311F12091BB01822F82958F7026
:1037E00090E002970CF460C08091B6019091B7010F
:1037F00098878F831986FB86EA862C87CE010796E9
:1038000051C0E51731F14D875E878D859E856A8BA6
:103810000E944C1A6A8981112EC0C8010E94321779
:10382000A4C08F2F807F69F77E2DF98AE88A898965
:103830000E94711A86EB91E00E943217E6EBF1E0EC
:1038400086E0DF011D928A95E9F70E94B11AD12C1A
:10385000DBC07413D8CF6111D6CFD8011596FC9375
:10386000C8010E943217E6EBF1E086E0DF011D920D
:103870008A95E9F7C9C0D62E662379F22091BB015B
:10388000822F82958F7090E0029774F08091B6013C
:103890009091B7019A8389831B82FD82EC822E83EB
:1038A000CE0101960E94321786E0F801A6EBB1E046
:1038B00001900D928A95E1F70E94BF1A6FC0E2163F
:1038C000F30628F0C701821B930B9C0104C02095CE
:1038D00030952E0D3F1D283C310508F052C0D62EE4
:1038E000662309F49ACFE5132CC074132AC0809183
:1038F000BB0180FD1DC0982F92959F70C9F0D80123
:1039000015968C9315979F3039F09F5F9295907F15
:103910008F70892B15968C93C8010E94321786E010
:10392000F801A6EBB1E001900D928A95E1F736C05F
:1039300086E0F801A6EBB1E001900D928A95E1F7DF
:1039400063C04D875E878D859E850E944C1A8823B3
:1039500079F086E0F801A6EBB1E001900D928A952E
:10396000E1F70E94BF1A0E94B11ADD24D3944CC023
:103970008091BB0181608093BB01C8010E94321716
:1039800043C07E2DF98AE88A89890E94711AE6EB84
:10399000F1E086E0DF011D928A95E9F70E94B11AF5
:1039A00033C0662309F439CF4D875E878D859E85A8
:1039B0000E944C1A882309F430CFCBCF4D875E8705
:1039C0008D859E850E94711F292F22952F7030E0D2
:1039D000223031052CF49F7041F0811106C00CC0DB
:1039E000243031052CF49F7049F4805E883020F03B
:1039F000C8010E943217CF2CDC2C06C0D8011596C6
:103A00009C91907F91F7F8CF8D2D62960FB6F89428
:103A1000DEBF0FBECDBFDF91CF911F910F91FF9001
:103A2000EF90DF90CF9008951F93CF93DF93CDB7A2
:103A3000DEB72C970FB6F894DEBF0FBECDBF4F8315
:103A4000588769877A878B879C87CE0107960E9463
:103A5000271B8823C1F02F8138858A859B85892B78
:103A600031F03F3F11F080E003C02F3FE1F781E0EC
:103A7000811147C04F81588569857A858B859C85E2
:103A80000E94801A3EC086E0FE013796DE01119644
:103A900001900D928A95E1F7FF81E8854A855B8563
:103AA0004115510531F0EF3F31F481E0FF3F19F44A
:103AB00003C081E001C080E080FD23C0209185012A
:103AC00030E0C9010196877099276091840170E008
:103AD00086179707F1F1F983EA835D834C8396E0BB
:103AE000929FD001939FB00D1124AA57BE4FFE01A3
:103AF000319601900D929A95E1F7809385010E948D
:103B0000901A16E08091840190918501891779F1CE
:103B1000189FC00111248A579E4F0E94271B88239B
:103B200031F1E09184011E9FF0011124EA57FE4F0C
:103B30004081518162817381848195810E94801AC4
:103B40008091840190E00196877099278093840189
:103B5000D9CF0E94481A1092850110928401E6EB99
:103B6000F1E086E0DF011D928A95E9F7CACF2C9635
:103B70000FB6F894DEBF0FBECDBFDF91CF911F917E
:103B80000895EF92FF920F931F93CF93DF939C01C1
:103B9000009709F471C0F12CEE24E394E901219619
:103BA000F9018491843740F4843008F056C08130A4
:103BB00081F0823021F160C0853709F449C0C0F13D
:103BC0009CE7980F903708F057C08F770E94D51662
:103BD00046C089010E5F1F4FFE01849190E2980F4D
:103BE000983050F48770FE2D01C0FF0F8A95EAF7D8
:103BF0008F2F0E94662015C00E940D1614C08901E7
:103C00000E5F1F4FFE01849190E2980F983068F488
:103C10008770FE2D01C0FF0F8A95EAF78F2F0E9453
:103C20006C200E948F20E8011AC00E94D516FBCF9D
:103C30002E5F3F4FFE01C491CC2341F08FE99FE0FE
:103C40000197F1F700C00000C150F6CFE90107C0AD
:103C5000FE01F490E901229602C00E940D168F2DFC
:103C6000882341F0EFE9FFE03197F1F700C0000051
:103C70008150F6CF9E0192CFDF91CF911F910F918E
:103C8000FF90EF90089508956093C0017093C10173
:103C90008093C2019093C3010C94361A0F931F9323
:103CA0000091C0011091C1012091C2013091C30166
:103CB000062B172B282B392B0093C0011093C10121
:103CC0002093C2013093C3011F910F910C94361AB7
:103CD0000F931F930091C0011091C1012091C20167
:103CE0003091C30106231723282339230093C001F1
:103CF0001093C1012093C2013093C3011F910F9112
:103D00000C94361A0F931F930091C0011091C101BA
:103D10002091C2013091C301062717272827392790
:103D20000093C0011093C1012093C2013093C301DD
:103D30001F910F910C94361A1092BC011092BD0184
:103D40001092BE011092BF010C94361A41E050E06F
:103D500060E070E004C0440F551F661F771F8A950E
:103D6000D2F74093BC015093BD016093BE017093A4
:103D7000BF010C94361A41E050E060E070E004C0EE
:103D8000440F551F661F771F8A95D2F78091BC019B
:103D90009091BD01A091BE01B091BF01842B952BE4
:103DA000A62BB72B8093BC019093BD01A093BE01BD
:103DB000B093BF010C94361A41E050E060E070E02F
:103DC00004C0440F551F661F771F8A95D2F7409590
:103DD0005095609570958091BC019091BD01A09126
:103DE000BE01B091BF0184239523A623B7238093FE
:103DF000BC019093BD01A093BE01B093BF010C9490
:103E0000361A41E050E060E070E004C0440F551FF6
:103E1000661F771F8A95D2F78091BC019091BD01F2
:103E2000A091BE01B091BF0184279527A627B7278F
:103E30008093BC019093BD01A093BE01B093BF01DC
:103E40000C94361A0F931F930091BC011091BD0181
:103E50002091BE013091BF01062B172B282B392B47
:103E60000093BC011093BD012093BE013093BF01AC
:103E70001F910F910C94361A0F931F930091BC0160
:103E80001091BD012091BE013091BF01062317237F
:103E9000282339230093BC011093BD012093BE0158
:103EA0003093BF011F910F910C94361A0F931F93FB
:103EB0000091BC011091BD012091BE013091BF0164
:103EC00006271727282739270093BC011093BD0127
:103ED0002093BE013093BF011F910F910C94361AAD
:103EE0000895CF92DF92EF92FF920F931F93CF939B
:103EF000DF93EC01C090C001D090C101E090C201FD
:103F0000F090C3018091BC019091BD01A091BE01D0
:103F1000B091BF01C82AD92AEA2AFB2A0FE110E092
:103F2000B701A601002E04C0769567955795479571
:103F30000A94D2F740FF07C0BE01802F0E94830B76
:103F40008130910539F40150110950F7BE0180E02C
:103F50000E94830BDF91CF911F910F91FF90EF9003
:103F6000DF90CF90089590910C01992361F1909189
:103F70000D01992341F1982F9695969596959F302E
:103F800088F4E0910E01F0910F01E90FF11D8770A7
:103F900021E030E001C0220F8A95EAF78181822B6F
:103FA000818308959091D70190FF2DC01F928F9328
:103FB0008BE295E09F938F930E9498070F900F904C
:103FC0000F900F90089540910E0150910F0120E045
:103FD00030E09FEFFA01E20FF31F6281681799F05A
:103FE0009F3F19F4611101C0922F2F5F3F4F2E3078
:103FF000310581F79F3F39F0FA01E90FF11D97FD77
:10400000FA9582830895089590910C01992369F19E
:1040100090910D01992349F1982F96959695969533
:104020009F3090F4E0910E01F0910F01E90FF11D26
:10403000877021E030E001C0220F8A95EAF72095D1
:1040400081812823218308959091D70190FF1FC07B
:104050001F928F938DE095E09F938F930E94980716
:104060000F900F900F900F90089540910E01509176
:104070000F0120E030E0FA01E20FF31F9281981364
:1040800001C012822F5F3F4F2E303105A1F70895F6
:1040900081E090E0E0910E01F0910F01E80FF91F2F
:1040A0001082019680319105A9F708959091D6016B
:1040B000982B9093D601089580959091D6019823DE
:1040C0009093D60108951092D60108959091D5014C
:1040D000982B9093D501089580959091D5019823C0
:1040E0009093D50108951092D50108958093C4014D
:1040F00008951092C401089540910E0150910F014E
:1041000020E030E080E0FA01E20FF31F918191118D
:104110008F5F2F5F3F4F2F303105A9F70895E09152
:104120000E01F0910F018091D6018083E0910E0184
:10413000F0910F0180819091D501892B808390911E
:10414000C401992361F0E0910E01F0910F0180818B
:10415000892B80830E947C2081111092C401809160
:104160000E0190910F010C948F1490933B0180935A
:104170003A010895CF92DF92EF92FF920F931F932F
:104180006C01EE24FF24C114D104E104F10421F4F4
:104190006B017C0180E001C080E133272F2D1E2DB3
:1041A0000D2D011511052105310519F0885F6801F4
:1041B000790197018601A4E0369527951795079513
:1041C000AA95D1F7011511052105310519F08C5F6C
:1041D0006801790197018601F2E0369527951795D8
:1041E0000795FA95D1F7011511052105310519F04B
:1041F0008E5F68017901B701A6017695679557959D
:104200004795452B462B472B09F08F5F1F910F9148
:10421000FF90EF90DF90CF9008958295982F9C7C2F
:1042200096959695837344E0849F90011124922B78
:10423000892F8A7A86959575990F892B08951F93F2
:10424000CF93DF931F92CDB7DEB799830E940D21E4
:10425000182F9981892F0E940D21212F30E0322FB4
:104260002227A901482BCA010F90DF91CF911F91FE
:1042700008958091F001843009F11092D80120E472
:1042800088E190E00FB6F894A895809360000FBE87
:104290002093600083B7817F846083BF83B7816090
:1042A00083BF7894889583B78E7F83BF88E10FB6EC
:1042B000F89480936000109260000FBE08950895F6
:1042C0000895CF930E945F210E9429090E946021D6
:1042D000C0E08C2F0E94540A811105C0CF5FCE3000
:1042E000C1F780E001C081E0CF9108950C94481A95
:1042F00082E084BD93E095BD9AEF97BD80936E00F8
:1043000008952FB7F8948091D9019091DA01A09186
:10431000DB01B091DC012FBF0895CF92DF92EF92C5
:10432000FF920F931F932FB7F8944091D9015091AA
:10433000DA016091DB017091DC012FBF6A017B0122
:10434000EE24FF248C0120E030E0C016D106E20606
:10435000F30610F441505109481B590BCA011F9133
:104360000F91FF90EF90DF90CF9008951F920F92E2
:104370000FB60F9211248F939F93AF93BF938091A9
:10438000D9019091DA01A091DB01B091DC01019695
:10439000A11DB11D8093D9019093DA01A093DB0197
:1043A000B093DC01BF91AF919F918F910F900FBEA1
:1043B0000F901F9018950E948A11F8942FEF87EAAA
:1043C00091E6215080409040E1F700C0000087E076
:1043D00090EBDC018093F9019093FA01A093FB012B
:1043E000B093FC012CE088E190E00FB6F894A8951A
:1043F000809360000FBE20936000FFCFEF92FF928A
:104400000F931F93CF93DF93E82EF12C8F2D0E94F3
:10441000540AC0E0D0E0082F10E098010C2E02C032
:10442000359527950A94E2F720FD05C02196C63000
:10443000D10599F709C06C2F7F2D80E00E94610B98
:10444000E812F4CF81E005C0F3948EE0F812DECFDD
:1044500080E0DF91CF911F910F91FF90EF90089531
:10446000CF93C82F8CE20E94FE21882321F08C2F4D
:10447000CF910C94FE2180E0CF910895CF930E94BC
:104480008B23811102C00E94712380E595E00E9478
:10449000FF06C5E6C15049F00E9429098FE39CE957
:1044A0000197F1F700C00000F5CF89E495E00E9484
:1044B000FF0689E20E943022811111C18AE20E9426
:1044C000302281110E94712385E00E9430228111E7
:1044D0000E94DB210E9496238093D70187E00E94EF
:1044E0003022882399F18BE10E943022882351F0F9
:1044F0009091D70191FB882780F921E0822780FBEA
:1045000091F922C08EE00E943022882351F09091D0
:10451000D70192FB882780F921E0822780FB92F95E
:1045200013C080E10E9430229091D701882341F08E
:1045300093FB882780F921E0822780FB93F904C050
:10454000892F809580FB90F99093D7018091D701B6
:104550000E949A230E94A8238093EA0180EE0E9481
:104560003022882341F08091EA01982F909590FBAA
:1045700080F98093EA0189E30E943022882359F070
:104580009091EA0191FB882780F921E0822780FB46
:1045900091F99093EA0182EE0E943022882359F02B
:1045A0009091EA0192FB882780F921E0822780FB25
:1045B00092F99093EA0186EE0E943022882359F006
:1045C0009091EA0193FB882780F921E0822780FB04
:1045D00093F99093EA0183EE0E943022882359F0E8
:1045E0009091EA0194FB882780F921E0822780FBE3
:1045F00094F99093EA0185E30E943022882359F0D0
:104600009091EA0195FB882780F921E0822780FBC1
:1046100095F99093EA0181E30E943022882359F0B2
:104620009091EA0196FB882780F921E0822780FBA0
:1046300096F99093EA0181E10E943022882359F093
:104640009091EA0197FB882780F921E0822780FB7F
:1046500097F99093EA018091EA010E94AC2380913E
:10466000EA0187FB882780F980930D0187E20E9489
:104670003022C82F8EE10E9430228111C2608FE16A
:104680000E9430228111C46080E20E943022811198
:10469000C86081E20E9430228111C06182E20E94E2
:1046A00030228111C06283E20E9430228111C064F5
:1046B00084E20E943022882311F0C06802C0CC231B
:1046C00029F08C2F0E94A3236C2F03C00E949F23EC
:1046D000682F70E080E090E0CF910C94441ECF9161
:1046E00008956DEE7EEF80E090E00E94662D60E020
:1046F00082E090E00E94582D60E083E090E00E940C
:10470000582D60E084E090E00E94582D60E085E044
:1047100090E00C94582D80E090E00E94522D21E012
:104720008D3E9E4F09F020E0822F089582E090E0B8
:104730000C944A2D682F82E090E00C94582D83E071
:1047400090E00C944A2D682F83E090E00C94582D53
:1047500084E090E00C944A2D682F84E090E00C9463
:10476000582D8091DF0180FF0BC06091130185E01F
:10477000689FB001112475956795759567952AC056
:1047800081FF09C06091130185E0689FB001112489
:10479000759567951FC082FF07C06091130185E082
:1047A000689FB001112416C04091E0014423C9F074
:1047B00060911201461788F72091130185E0289F28
:1047C00090011124429FC001439F900D112470E07D
:1047D0000E941C2D6038710540F46115710539F097
:1047E00002C065E070E0862F08958FE7089581E0AC
:1047F00008958091DF0180FF08C06091110170E091
:10480000759567957595679521C081FF06C0609184
:10481000110170E07595679519C082FF04C0609121
:10482000110170E010C08091E0018823C1F0609117
:1048300010018617A0F790911101989FC0011124D3
:1048400070E00E941C2D6038710528F46115710517
:1048500021F0862F08958FE7089581E0089561E0A3
:1048600070E0F4CF803F21F40E94B123819504C011
:10487000813F29F40E94B1238093E3010895823F90
:1048800021F40E94B123819504C0833F29F40E9442
:10489000B1238093E2010895893F19F40E94F9231E
:1048A00005C08A3F31F40E94F92381958093E40189
:1048B00008958B3F21F40E94F923819504C08C3F19
:1048C00029F40E94F9238093E5010895843F21F49F
:1048D0008091E101816017C0853F21F48091E10161
:1048E000826011C0863F21F48091E10184600BC099
:1048F000873F21F48091E101886005C0883F31F451
:104900008091E10180618093E10108958D3F21F460
:104910008091DF0181600BC08E3F21F48091DF0127
:10492000826005C08F3F29F48091DF01846080930D
:10493000DF010895803F39F48091E30187FF6CC067
:104940001092E30169C0813F29F48091E3011816B8
:10495000BCF362C09091E201823F29F497FF5CC0F2
:104960001092E20159C0833F19F41916CCF354C0D8
:10497000893F41F48091E40118160CF04DC010926B
:10498000E4014AC08A3F29F48091E40187FF44C0D2
:10499000F6CF8B3F39F48091E50187FF3DC010923F
:1049A000E5013AC08C3F29F48091E5011816BCF36B
:1049B00033C0843F21F48091E1018E7F17C0853F91
:1049C00021F48091E1018D7F11C0863F21F4809117
:1049D000E1018B7F0BC0873F21F48091E101877F4C
:1049E00005C0883F31F48091E1018F7E8093E10121
:1049F00013C08D3F21F48091DF018E7F0BC08E3F6D
:104A000021F48091DF018D7F05C08F3F29F48091D3
:104A1000DF018B7F8093DF018091E20181110EC065
:104A20008091E30181110AC08091E401811106C0E7
:104A30008091E501811102C01092E00108958091FA
:104A4000D70183FF7EC08CE895E00E94FF0680912D
:104A5000E1011F928F9387E895E09F938F930E94C7
:104A6000980785E895E00E94FF062091E201822FD9
:104A7000992787FD90959F932F9382E895E09F93C8
:104A80008F930E94980780E895E00E94FF0620918E
:104A9000E301822F992787FD90959F932F938DE7B0
:104AA00095E09F938F930E9498078BE795E00E9473
:104AB000FF062091E401822F992787FD90959F930F
:104AC0002F9388E795E09F938F930E94980786E73E
:104AD00095E00E94FF062091E501822F992787FD2E
:104AE00090959F932F9383E795E09F938F930E94D8
:104AF000980780E795E00E94FF068091E0011F92F1
:104B00008F938DE695E09F938F930E9498078BE695
:104B100095E00E94FF068091DF011F928F9388E647
:104B200095E09F938F930E94980785E695E00E94F9
:104B3000FF068DB79EB74C960FB6F8949EBF0FBE7A
:104B40008DBF81EE91E00E94D4140E948121909348
:104B5000DE018093DD0108951F93CF93DF93809151
:104B6000DD019091DE010E948D214091E0014423FE
:104B700021F02091140130E006C0209115015AE087
:104B8000259F900111248217930708F482C0809119
:104B9000E2011091E301D091E401C091E50181119E
:104BA00007C0111105C0D11103C0CC2309F471C095
:104BB0004F3F19F04F5F4093E001181624F40E9414
:104BC000B1238093E2018091E20187FF05C00E943A
:104BD000B12381958093E201111624F40E94B12340
:104BE0008093E3018091E30187FF05C00E94B12318
:104BF00081958093E3016091E201662339F1109180
:104C0000E301112319F1772767FD7095872F972FFF
:104C10000E94212C23E333E343E35FE30E94852CCE
:104C20000E94EE2B6093E201612F772767FD70955C
:104C3000872F972F0E94212C23E333E343E35FE385
:104C40000E94852C0E94EE2B6093E3011D1624F434
:104C50000E94F9238093E4018091E40187FF05C05D
:104C60000E94F92381958093E4011C1624F40E948C
:104C7000F9238093E5018091E50187FF05C00E943B
:104C8000F92381958093E501DF91CF911F910C94D9
:104C90001F25DF91CF911F910895E1EEF1E085E0AE
:104CA000DF011D928A95E9F71092E0011092DF0171
:104CB00008958FEA97E00E94FF061F9281E08F938C
:104CC0001F9285E08F9381E697E09F938F930E94D8
:104CD00098070F900F900F900F900F900F900895DE
:104CE0008330E9F128F4813061F0823009F10895D0
:104CF000853009F462C008F449C0863009F474C0F4
:104D0000089520911501862F90E0820F911D8F3F0D
:104D1000910520F4620F6093150103C08FEF80931B
:104D20001501809115011F928F938AE996E072C058
:104D300020911401862F90E0820F911D8F3F9105E5
:104D400020F4620F6093140103C08FEF809314016D
:104D5000809114011F928F9388E896E05BC02091A8
:104D60001301862F90E0820F911D8F3F910520F453
:104D7000620F6093130103C08FEF80931301809142
:104D800013011F928F9385E796E044C02091120192
:104D9000862F90E0820F911D8F3F910520F4620FC6
:104DA0006093120103C08FEF809312018091120172
:104DB0001F928F9380E696E02DC020911101862FDF
:104DC00090E0820F911D8F3F910520F4620F609358
:104DD000110103C08FEF80931101809111011F9287
:104DE0008F9387E496E016C020911001862F90E003
:104DF000820F911D8F3F910520F4620F6093100187
:104E000003C08FEF80931001809110011F928F9348
:104E10008CE296E09F938F930E9498070F900F90DB
:104E20000F900F900895833081F128F4813059F06C
:104E30008230D1F00895853009F449C0B8F1863048
:104E400009F456C0089580911501681720F4861B57
:104E50008093150102C010921501809115011F92D7
:104E60008F938DE196E054C080911401681720F46F
:104E7000861B8093140102C01092140180911401CA
:104E80001F928F938BE096E043C0809113016817C7
:104E900020F4861B8093130102C0109213018091AD
:104EA00013011F928F9388EF95E032C08091120119
:104EB000681720F4861B8093120102C01092120121
:104EC000809112011F928F9383EE95E021C0809113
:104ED0001101681720F4861B8093110102C0109203
:104EE0001101809111011F928F938AEC95E010C0FF
:104EF00080911001681720F4861B8093100102C076
:104F000010921001809110011F928F938FEA95E00B
:104F10009F938F930E9498070F900F900F900F9080
:104F20000895CF93C82F1F928F9324EB38E03F93BF
:104F30002F930E94980761E070E080E090E004C049
:104F4000660F771F881F991FCA95D2F70E94441ECB
:104F50000F900F900F900F90CF910C94481ACF9311
:104F60008D3109F465C0B0F58E3009F4CBC100F580
:104F7000873009F49BC1A8F4863009F06AC2809199
:104F8000D701817F8E7F8093D70189EB98E00E94C3
:104F9000FF068BEF9CE00E94FF0681E08093E70113
:104FA00080C1883009F44FC08B3009F47CC151C2F4
:104FB000863109F4EDC138F4803109F4B6C181318C
:104FC00009F42DC246C2893109F4CBC18B3109F4F1
:104FD00086C13FC2853309F434C248F4873209F4EC
:104FE00030C208F430C2893209F42BC232C2833491
:104FF00038F48A3308F029C2883309F454C129C22D
:10500000833409F41EC2883409F023C20E94481A6E
:105010008AEE9CE00E94FF069FEF23ED80E3915013
:1050200020408040E1F700C000000E94DB2139C130
:105030008AE09DE00E94FF060E94A82B0E94831434
:105040000E94C10C2EC18FEF9CE00E94FF068AECEB
:105050009AE00E94FF060E949F231F928F9387EC85
:105060009AE09F938F930E94980785EC9AE00E94A4
:10507000FF060E949623C82F82EB9AE00E94FF064B
:105080001F92CF932DEA3AE03F932F930E94980707
:105090008BEA9AE00E94FF0681EA9AE00E94FF06EE
:1050A0008C2F81701F928F932EE93AE03F932F93BC
:1050B0000E9498078CE99AE00E94FF0682E99AE034
:1050C0000E94FF06C1FB882780F91F928F932FE86B
:1050D0003AE03F932F930E9498078DE89AE00E9450
:1050E000FF0681E89AE00E94FF06C2FB882780F94C
:1050F0001F928F932EE73AE03F932F930E949807D9
:105100008CE79AE00E94FF0683E79AE00E94FF0680
:10511000C3FBCC27C0F91F92CF9380E79AE09F93FF
:105120008F930E9498078EE69AE00E94FF060E94E5
:10513000A823C82F8AE59AE00E94FF061F92CF930A
:1051400025E53AE03F932F930E94980783E59AE084
:105150000E94FF068AE39AE00E94FF068C2F81706E
:105160001F928F9327E33AE03F932F930E94980773
:105170008DB79EB780960FB6F8949EBF0FBE8DBFB9
:1051800085E39AE00E94FF068EE19AE00E94FF0606
:10519000C1FB882780F91F928F932BE13AE03F9360
:1051A0002F930E94980789E19AE00E94FF0687E00A
:1051B0009AE00E94FF06C2FB882780F91F928F9316
:1051C00024E03AE03F932F930E94980782E09AE010
:1051D0000E94FF0680EF99E00E94FF06C3FB88272C
:1051E00080F91F928F932DEE39E03F932F930E9409
:1051F00098078BEE99E00E94FF0681EE99E00E94ED
:10520000FF06C4FB882780F91F928F932EED39E0AB
:105210003F932F930E9498078CED99E00E94FF0620
:105220008AEC99E00E94FF06C5FB882780F91F924F
:105230008F9327EC39E03F932F930E94980785ECDA
:1052400099E00E94FF0689EA99E00E94FF06C6FBEA
:10525000882780F91F928F9326EA39E03F932F9396
:105260000E94980784EA99E00E94FF068CE999E081
:105270000E94FF06C7FBCC27C0F91F92CF9389E994
:1052800099E09F938F930E94980787E999E00E9485
:10529000FF068DB79EB74C960FB6F8949EBF0FBE13
:1052A0008DBFC1E0DBC080EE98E058C08091D7018F
:1052B000C82FC17080FF09C08DED9CE00E94FF06E1
:1052C0008091D701817F8E7F44C081ED9CE00E9458
:1052D000FF068091D70181608093D701E2CF809152
:1052E000D70181FBCC27C0F991E0C927C0FB81F928
:1052F0008093D701CC2319F084EC9CE025C086EB89
:105300009CE02CC08091D70182FBCC27C0F991E0B2
:10531000C927C0FB82F98093D701CC2319F087EA13
:105320009CE012C087E99CE019C08091D70183FB03
:10533000CC27C0F991E0C927C0FB83F98093D7013E
:10534000CC2351F08BE89CE00E94FF068091D701AE
:1053500081608093D70182C08EE79CE00E94FF06A7
:10536000A0CF8FE69CE00E94FF0683E49CE00E94B1
:10537000FF0686E09CE00E94FF0689ED9BE00E940C
:10538000FF0685E99BE00E94FF068AE69BE0E6CFE8
:105390008CE59BE00E94FF060E9483141F928F936E
:1053A00082E49BE09F938F930E94980780910C0169
:1053B0001F928F938BE29BE09F938F930E9498079D
:1053C00080916E011F928F9388E19BE09F938F9352
:1053D0000E94980780910D011F928F9385E09BE0BA
:1053E0009F938F930E9498078091D9019091DA0141
:1053F000A091DB01B091DC01BF93AF939F938F939A
:1054000081EF9AE09F938F930E9498078DB79EB784
:1054100046960FB6F8949EBF0FBE8DBF42CF0E9436
:10542000481AC0910D0181E0C827C0930D01CC231B
:1054300029F087EE9AE00E94FF0610C08CED9AE0FA
:105440008DCF80E003C08D5101C089530E94912708
:1054500028CF8AED9AE00E94FF06C0E08C2FCF9102
:10546000089580E0089580E00895CF93C82F80913B
:10547000E701813081F020F0823009F44CC042C154
:10548000A0910E01B0910F018C91813169F08232AF
:1054900009F03AC109C0A0910E01B0910F018C91A1
:1054A000813111F0823249F48C2F0E94312A81110E
:1054B0002FC08C2F0E94AF272CC08C2F0E94332A24
:1054C000811126C0C431E1F070F4CB3081F0C031DD
:1054D000D1F40E9459268CEA98E00E94FF0682E0EF
:1054E0008093E70115C0C93259F0C83361F489EBE4
:1054F00098E00E94FF0680EB98E00E94FF0608C03B
:105500001092E70103C18AEA98E00E94FF06FEC0FC
:1055100081E08170FDC0C43220F5CE3108F0C0C0FA
:10552000CB3099F1C8F4C73009F0D2C08AE080933B
:10553000150194E19093140193E0909313018093EB
:10554000120188E08093110188E28093100180E5C8
:1055500097E00E94FF06BFC0C33149F1C431C1F0DA
:10556000B7C0CB3409F4A9C028F4C93289F0C833D4
:1055700061F0AEC0C13509F49EC0C23509F499C0CE
:10558000CE3409F0A5C06AE09EC00E945926A3C08F
:105590008091E601882319F01092E6019CC08DE508
:1055A00097E00E94FF0681E08093E701B1C087E3A6
:1055B00097E00E94FF0685E297E00E94FF06809137
:1055C00015011F928F9382E297E09F938F930E9421
:1055D000980780E297E00E94FF068EE097E00E9425
:1055E000FF06809114011F928F938BE097E09F93A9
:1055F0008F930E94980789E097E00E94FF068AEF48
:1056000096E00E94FF06809113011F928F9387EF0F
:1056100096E09F938F930E94980785EF96E00E94F3
:10562000FF0684EE96E00E94FF06809112011F9211
:105630008F9381EE96E09F938F930E9498078FED52
:1056400096E00E94FF068AEC96E00E94FF06809199
:1056500011011F928F9387EC96E09F938F930E9486
:10566000980785EC96E00E94FF068EEA96E00E947D
:10567000FF06809110011F928F938BEA96E09F9313
:105680008F930E94980789EA96E00E94FF068DB7E3
:105690009EB748960FB6F8949EBF0FBE8DBF1BC035
:1056A000CE51EC2FF0E0E15DFE4F80818093E6016A
:1056B00012C061E003C061E006C06AE08091E601CB
:1056C0000E94702608C08091E6010E94132703C043
:1056D0008EE497E013C08091E601882369F01F9261
:1056E0008F9388E497E09F938F930E9498070F9081
:1056F0000F900F900F9004C085E497E00E94FF0682
:1057000081E006C01092E70180E002C080E001CF96
:10571000CF910895E1E8F0E0808188608083808106
:10572000816080838FB7F89493E09093890090ED27
:10573000909388008FBF0895EFE6F0E0808182604B
:1057400080830895EFE6F0E080818D7F8083089567
:10575000EFE6F0E0808192E08927808308951F9230
:105760000F920FB60F9211242F933F934F935F9395
:105770006F937F938F939F93AF93BF93EF93FF9319
:105780008091E8019091E90101969093E90180935D
:10579000E801811103C082E00E94C10CE091E9019F
:1057A000E695E695F0E0E65EF24FE4918091E8013F
:1057B0008E1303C080E00E94C10CFF91EF91BF9156
:1057C000AF919F918F917F916F915F914F913F9199
:1057D0002F910F900FBE0F901F90189504D06894D2
:1057E000B1118DC0089570D088F09F5790F0B92FF7
:1057F0009927B751A0F0D1F0660F771F881F991F26
:105800001AF0BA95C9F712C0B13081F077D0B1E083
:10581000089574C0672F782F8827B85F39F0B93F93
:10582000CCF3869577956795B395D9F73EF4909527
:105830008095709561957F4F8F4F9F4F0895E894A5
:1058400009C097FB3EF490958095709561957F4FC8
:105850008F4F9F4F9923A9F0F92F96E9BB27939576
:10586000F695879577956795B795F111F8CFFAF486
:10587000BB0F11F460FF1BC06F5F7F4F8F4F9F4FB7
:1058800016C0882311F096E911C0772321F09EE815
:10589000872F762F05C0662371F096E8862F70E07B
:1058A00060E02AF09A95660F771F881FDAF7880F55
:1058B0009695879597F9089557FD9058440F551F71
:1058C00059F05F3F71F04795880F97FB991F61F082
:1058D0009F3F79F087950895121613061406551FF9
:1058E000F2CF4695F1DF08C0161617061806991F65
:1058F000F1CF86957105610508940895E894BB275A
:1059000066277727CB0197F908950BD078C069D027
:1059100028F06ED018F0952309F05AC05FC011240A
:10592000EECFCADFA0F3959FD1F3950F50E0551F3E
:10593000629FF001729FBB27F00DB11D639FAA27E4
:10594000F00DB11DAA1F649F6627B00DA11D661F33
:10595000829F2227B00DA11D621F739FB00DA11D54
:10596000621F839FA00D611D221F749F3327A00D0E
:10597000611D231F849F600D211D822F762F6A2FAA
:1059800011249F5750408AF0E1F088234AF0EE0F2F
:10599000FF1FBB1F661F771F881F91505040A9F73C
:1059A0009E3F510570F014C0AACF5F3FECF3983EC4
:1059B000DCF3869577956795B795F795E7959F5FA3
:1059C000C1F7FE2B880F911D9695879597F908953D
:1059D00097F99F6780E870E060E008959FEF80ECA2
:1059E000089500240A941616170618060906089545
:1059F00000240A9412161306140605060895092EAB
:105A00000394000C11F4882352F0BB0F40F4BF2B19
:105A100011F460FF04C06F5F7F4F8F4F9F4F089559
:105A2000991B79E004C0991F961708F0961B881FF0
:105A30007A95C9F78095089597FB072E16F4009480
:105A400007D077FD09D00E94362D07FC05D03EF423
:105A5000909581959F4F0895709561957F4F08951A
:105A6000EE0FFF1F0590F491E02D0994AA1BBB1BBC
:105A700051E107C0AA1FBB1FA617B70710F0A61B4E
:105A8000B70B881F991F5A95A9F780959095BC016F
:105A9000CD010895F999FECF92BD81BDF89A99275D
:105AA00080B50895A8E1B0E042E050E00C946D2D7F
:105AB000262FF999FECF1FBA92BD81BD20BD0FB62A
:105AC000F894FA9AF99A0FBE019608950E94582DFB
:105AD000272F0C94592DDC01CB01FC01F999FECF45
:105AE00006C0F2BDE1BDF89A319600B40D92415066
:0A5AF0005040B8F70895F894FFCF76
:105AFA002002C20CB30D900D5C0D290D0101C501E8
:105B0A0028080A03140A3F4D3620399A044D04170F
:105B1A0004F703BE0331034A0363037C039C0301B6
:0A5B2A000203040506070809000045
:00000001FF
